:100000000C942A000C9445000C9445000C94450077
:100010000C9445000C9445000C9445000C9445004C
:100020000C9445000C9445000C9445000C9445003C
:100030000C9445000C9445000C9445000C9445002C
:100040000C9445000C9445000C9445000C9445001C
:100050000C94450011241FBECFE5D8E0DEBFCDBF14
:1000600010E0A0E6B0E0E8ECF0E002C005900D92F0
:10007000A036B107D9F710E0A0E6B0E001C01D92AC
:10008000A036B107E1F70C9456000C940000181646
:1000900019065CF4AC011816190624F49C012150D1
:1000A0003040E9F741505040B1F70895CFE5D8E02E
:1000B000DEBFCDBF8FEF8ABBC0E0CBBB88EE93E045
:0800C0000E944700CF5FF9CF59
:00000001FF
